:020000040000FA
:040000008431EB2C30
:080008002000233095002000C8
:10001000AB0A07302B020318AB012A14AC0F1328CC
:10002000AD0F1328AA14A6211830AE001430FF001B
:10003000FE0120008C018E0120002B080B002B28D4
:100040006828A528B228EF282C29692920008C01CE
:10005000200090120900C03084000030850015088F
:100060000002031C7E14B4308400003085001508A3
:100070000002031CFE14A83084000030850015081F
:100080000002031C7E15C130840000308500150875
:100090000002031CFE15B5308400003085001508F1
:1000A0000002031C7E16A93084000030850015086C
:1000B0000002031CFE1621007F088C007E088E00C3
:1000C000200020308C0000308E00AE0B2B2826281C
:1000D000A73084000030850015080002031CFF16BD
:1000E000BD3084000030850015080002031CFE149A
:1000F000B13084000030850015080002031C7E1515
:10010000A53084000030850015080002031CFE1590
:10011000BF3084000030850015080002031C7E16E5
:10012000B33084000030850015080002031CFE1661
:1001300021007F088C007E088E00200000308C009B
:1001400001308E00AE0B6828262821007F088C0025
:100150007E088E00200000308C0002308E00AE0B36
:10016000A5282628C230840000308500150800022A
:10017000031CFF16B630840000308500150800020D
:10018000031C7E14AA30840000308500150800028C
:10019000031CFE14C33084000030850015080002E3
:1001A000031CFE15B73084000030850015080002DE
:1001B000031C7E16AB308400003085001508000259
:1001C000031CFE1621007F088C007E088E00200094
:1001D00000308C0004308E00AE0BB2282628A630EA
:1001E00084000030850015080002031CFF16B8309B
:1001F00084000030850015080002031C7E14AC301A
:1002000084000030850015080002031CFE14A03095
:1002100084000030850015080002031C7E15BE30E6
:1002200084000030850015080002031C7E16B230E1
:1002300084000030850015080002031CFE16210012
:100240007F088C007E088E00200000308C00083073
:100250008E00AE0BEF282628AE30840000308500DB
:1002600015080002031CFF16A23084000030850030
:1002700015080002031C7E14B9308400003085008C
:1002800015080002031CFE14AD3084000030850008
:1002900015080002031C7E15A13084000030850083
:1002A00015080002031CFE15BA30840000308500DA
:1002B00015080002031CFE1621007F088C007E0832
:1002C0008E00200000308C0010308E00AE0B2C29E8
:1002D0002628BC3084000030850015080002031C6D
:1002E000FF16B03084000030850015080002031CA2
:1002F0007E14A43084000030850015080002031C21
:10030000FE14BB3084000030850015080002031C79
:100310007E15AF3084000030850015080002031CF4
:10032000FE15A33084000030850015080002031C70
:100330007E1621007F088C007E088E002000003091
:100340008C0020308E00AE0B69292628A0012000E9
:100350000C1EA0140C1D20150800AF00AF0BAE2919
:100360000800B0000000B00BB2290800B50A35083B
:10037000123C0319B5013508A200FD01FC0108007B
:10038000B5033508013E031DC8291130B500A20090
:10039000FD01FC0108002108B500A200EE3E031C8F
:1003A000D5291130B5023508CE29FD01FC01080020
:1003B000B1002A102A1CDA29B10BD9290800200023
:1003C000350AB800B701B901BA01BB01BC01383028
:1003D0004C18BB00FF30DC24FF30DC24FF30DC2471
:1003E000FF30DC2408008530870039308600350A6C
:1003F000B4001600B2001600B300B40BF92933089C
:1004000086003208B21787000800F0303202031D60
:10041000102A33087D072622FD0F112AFC0A112A13
:1004200016000800310015173100703092007D0869
:1004300091007B0893003100151555308B13960001
:10044000AA30960095148B172000080084007030A5
:100450008500003F080000302622CC0008002B2237
:100460004C1C342A4C10352A4C140030FD004C082A
:10047000FB001222DF21DF210800F321FD01FC0136
:100480000522B600B6130522CB00CB0A0522CD000B
:10049000231C662A07302402031D512ACB21A30105
:1004A0003D2AA408031D662A203021020319B62123
:1004B000213021020319C021003021020319B501A6
:1004C0000C30210203192F22A3013D2A200020080D
:1004D00003197F2ADF21DF21DF21DF2106302002FF
:1004E00003192F22A018772A20197B2A3D2AB6212A
:1004F000DF21DF216E2AC021DF21DF216E2A0F30AC
:1005000036020319A1221030360282310319BD22AE
:1005100082311130360203196023123036028331E2
:1005200003198E2382312508003E031D9E2AAA1C32
:100530009E2AAA104C1C9E2AB6213D2ACD0B482A81
:100540003D2A0522B7000522B8000522B900052280
:10055000BA000522BB000522BC00C0303705CE0022
:100560000310CE0CCE0CCE0CCE0CCE0CCE0CCE0A84
:100570004B08DC24CE0BB82A08000522B700052260
:10058000B8001F303705CF001F304F02031DD02A9F
:10059000B701B801B901BA01BB01BC01DC24E72AEB
:1005A000B71BD42AE822D52AFC22371BD92A1023CC
:1005B000DA2A2423B71ADE2A3823DF2A4C234B08F1
:1005C000D8212018E72A2318E72ACF0BD02A0800C1
:1005D0000B30D000AA3084000008840A8000840315
:1005E0008403D00BEC2A840A80014030381B80073A
:1005F000A030B81B800708000B30D000A130840069
:10060000000884038000840A840AD00B002B840332
:1006100080014030381B8007A030B81B80070800DD
:100620000B30D000B63084000008840A80008403B8
:100630008403D00B142B840A80014030381A8007C1
:10064000A030B81A800708000B30D000AD3084000D
:10065000000884038000840A840AD00B282B8403BA
:1006600080014030381A8007A030B81A800708008F
:100670000B30D000C23084000008840A800084035C
:100680008403D00B3C2B840A80014030381980074A
:10069000A030B819800708000B30D000B9308400B2
:1006A000000884038000840A840AD00B502B840342
:1006B0008001403038198007A030B8198007080041
:1006C0000522B7000522B8000522B9000522BA00AC
:1006D0000522BB000522BC000522BD000522BE008C
:1006E0000522BF000522C0000522C7000522C80060
:1006F0000522CE00CE0AB71B822B4B08DC24CE0B82
:100700007B2B080086315A2683314B08D8212018CC
:100710008D2B23188D2BCE0B7B2B080082310522CD
:10072000B7000522B8000522B9000522BA0005224B
:10073000BB000522BC008331CE01B71B4E14371B12
:10074000CE14B91B4E15391BCE15BB1B4E163B1BC9
:10075000CE16A0308400003085003818D424381C10
:10076000D824A130840000308500B818D424B81CE7
:10077000D824A2308400003085003819D424381DD4
:10078000D824A330840000308500B819D424B81DC3
:10079000D824A430840000308500381AD424381EB0
:1007A000D824A530840000308500B81AD424B81E9F
:1007B000D824A630840000308500381BD424381F8C
:1007C000D824A730840000308500B81BD424B81F7B
:1007D000D824A8308400003085003718D424371C72
:1007E000D824A930840000308500B718D424B71C61
:1007F000D824AA308400003085003719D424371D4E
:10080000D824AB30840000308500B719D424B71D3C
:10081000D824AC308400003085003A18D4243A1C27
:10082000D824AD30840000308500BA18D424BA1C16
:10083000D824AE308400003085003A19D4243A1D03
:10084000D824AF30840000308500BA19D424BA1DF2
:10085000D824B0308400003085003A1AD4243A1EDF
:10086000D824B130840000308500BA1AD424BA1ECE
:10087000D824B2308400003085003A1BD4243A1FBB
:10088000D824B330840000308500BA1BD424BA1FAA
:10089000D824B4308400003085003918D424391CA1
:1008A000D824B530840000308500B918D424B91C90
:1008B000D824B6308400003085003919D424391D7D
:1008C000D824B730840000308500B919D424B91D6C
:1008D000D824B8308400003085003C18D4243C1C57
:1008E000D824B930840000308500BC18D424BC1C46
:1008F000D824BA308400003085003C19D4243C1D33
:10090000D824BB30840000308500BC19D424BC1D21
:10091000D824BC308400003085003C1AD4243C1E0E
:10092000D824BD30840000308500BC1AD424BC1EFD
:10093000D824BE308400003085003C1BD4243C1FEA
:10094000D824BF30840000308500BC1BD424BC1FD9
:10095000D824C0308400003085003B18D4243B1CD0
:10096000D824C130840000308500BB18D424BB1CBF
:10097000D824C2308400003085003B19D4243B1DAC
:10098000D824C330840000308500BB19D424BB1D9B
:10099000D82481314B08D82183312018D32C231837
:1009A000D32CCE0BA92B0800800A0319800908005C
:1009B0008008031D80030800CA00A0308400243092
:1009C000D10000301A00D10BE22C85315D25843135
:1009D0004A08D82108008C019501B5010030B50006
:1009E000A501A901A401A101A601A701A801A301D4
:1009F000AB010430AB00AC01AD01A00120008030A0
:100A0000970020004230980023008C012100143010
:100A10008C0021008E0124008C010C150C16240082
:100A20008E012000A0010B172100901620008B17CB
:100A3000FF30B700B800B900BA00BB00BC00843179
:100A4000FF30DC24FF30DC242000B701B801B901FD
:100A5000BA01BB01BC01FF30DC24FF30DC24FF30D5
:100A6000DC242B222008B800FF30DC24FF30DC24FB
:100A70003D2A87347B34873496348734E134883494
:100A80002C348834BF34893464348934AF348A34A4
:100A900042348A34DB348C3494348C349D348C343A
:100AA000AC348C34D3348C34FA348D340F348D34EC
:100AB0002A348D3439348D344834A03084000030E9
:100AC0008500FF3038188000A13084000030850098
:100AD000FF30B8188000A230840000308500FF305D
:100AE00038198000A330840000308500FF30B81929
:100AF0008000A430840000308500FF30381A800068
:100B0000A530840000308500FF30B81A8000A63080
:100B1000840000308500FF30381B8000A73084003F
:100B200000308500FF30B81B8000A8308400003002
:100B30008500FF3037188000A93084000030850020
:100B4000FF30B7188000AA30840000308500FF30E5
:100B500037198000AB30840000308500FF30B719B2
:100B60008000AC30840000308500FF303A188000EF
:100B7000AD30840000308500FF30BA188000AE3000
:100B8000840000308500FF303A198000AF308400C7
:100B900000308500FF30BA198000B030840000308A
:100BA0008500FF303A1A8000B130840000308500A3
:100BB000FF30BA1A8000B230840000308500FF3068
:100BC0003A1B8000B330840000308500FF30BA1B30
:100BD0008000B430840000308500FF303918800078
:100BE000B530840000308500FF30B9188000B63081
:100BF000840000308500FF3039198000B730840050
:100C000000308500FF30B9198000B8308400003012
:100C10008500FF303C188000B9308400003085002A
:100C2000FF30BC188000BA30840000308500FF30EF
:100C30003C198000BB30840000308500FF30BC19B7
:100C40008000BC30840000308500FF303C1A8000FA
:100C5000BD30840000308500FF30BC1A8000BE30FB
:100C6000840000308500FF303C1B8000BF308400D2
:100C700000308500FF30BC1B8000C0308400003095
:100C80008500FF303B188000C130840000308500B3
:100C9000FF30BB188000C230840000308500FF3078
:100CA0003B198000C330840000308500FF30BB1941
:100CB00080000800A0308400003085003818800AC9
:100CC0003E188003A130840000308500B818800AE7
:100CD000BE188003A2308400003085003819800AD5
:100CE0003E198003A330840000308500B819800AC3
:100CF000BE198003A430840000308500381A800AB1
:100D00003E1A8003A530840000308500B81A800A9E
:100D1000BE1A8003A630840000308500381B800A8C
:100D20003E1B8003A730840000308500B81B800A7A
:100D3000BE1B8003A8308400003085003718800A6D
:100D40003D188003A930840000308500B718800A60
:100D5000BD188003AA308400003085003719800A4E
:100D60003D198003AB30840000308500B719800A3C
:100D7000BD198003AC308400003085003A18800A29
:100D800040188003AD30840000308500BA18800A16
:100D9000C0188003AE308400003085003A19800A04
:100DA00040198003AF30840000308500BA19800AF2
:100DB000C0198003B0308400003085003A1A800AE0
:100DC000401A8003B130840000308500BA1A800ACE
:100DD000C01A8003B2308400003085003A1B800ABC
:100DE000401B8003B330840000308500BA1B800AAA
:100DF000C01B8003B4308400003085003918800A9D
:100E00003F188003B530840000308500B918800A8F
:100E1000BF188003B6308400003085003919800A7D
:100E20003F198003B730840000308500B919800A6B
:100E3000BF198003B8308400003085003C18800A58
:100E400048188003B930840000308500BC18800A3F
:100E5000C8188003BA308400003085003C19800A2D
:100E600048198003BB30840000308500BC19800A1B
:100E7000C8198003BC308400003085003C1A800A09
:100E8000481A8003BD30840000308500BC1A800AF7
:100E9000C81A8003BE308400003085003C1B800AE5
:100EA000481B8003BF30840000308500BC1B800AD3
:100EB000C81B8003C0308400003085003B18800AC6
:100EC00047188003C130840000308500BB18800AB9
:100ED000C7188003C2308400003085003B19800AA7
:100EE00047198003C330840000308500BB19800A95
:100EF000C719800308001034FF340C341F34003449
:100F00008D34C0341F3400340D34C0341F340034E9
:100F10004D3430341F3400340D3430341F34003439
:100F20002D340C341F3400340D340C34123404349A
:100F30000C34C034FF34CF34F034CF340F34C834E1
:100F40007F34CF34F834CF348734CC343F34C73493
:100F5000FC34CF34C334CE341F34C334FE34CF34E6
:100F6000E134CF340F34C034FF34CF34F034CF34D5
:100F70008734C8347F34C734F834CF34C334CC34E6
:100F80003F34C334FC34CF34E134CE341F34C13465
:100F9000FE34CF34F034CF340F34C034FF34C73490
:100FA000F834CF348734C8347F34C334FC34CF347E
:100FB000C334CC343F34C134FE34CF34E134CE3486
:100FC0001F34123404340C34C034FF34CE341F3494
:100FD000CF344334C8347F34CC343F34CF34E1345D
:100FE000CC343F34C8347F34CF34F034CE341F3463
:100FF000C034FF34C734F834CF340F34C134FE3436
:10100000C334FC34CF348734C334FC34C134FE34AD
:10101000CF34C334C734F834C034FF34CF34E13470
:10102000CF34F034C8347F34CF34F034CF34E134AB
:10103000CC343F34C734F834CF34C334CE341F34C7
:10104000C334FC34CF348734CF340F34C134FE344E
:10105000CF340F34CF340734123404341834FF340F
:10106000FF34C0340034C0340034FF34FF34C034A3
:101070000034C0340034FF34FF34C0340034C03492
:101080000034FF34FF34C0340034C0340034C03482
:101090000034C0340034C0340034C0340034C034B0
:1010A0000034C0340034C0340034C0340034C034A0
:1010B0000034C0340034C0340034C0340034C03490
:1010C0000034FF34FF34C0340034C0340034FF3403
:1010D000FF34C0340034C0340034FF34FF34C03433
:1010E0000034C0340034FF34FF34C0340034C03422
:1010F0000034C0340034C0340034C0340034C03450
:101100000034C0340034C0340034C0340034C0343F
:101110000034C0340034C0340034C0340034C0342F
:101120000034C0340034FF34FF34C0340034C034E1
:101130000034FF34FF34C0340034C0340034FF3492
:10114000FF34C0340034C0340034FF34FF34C034C2
:101150000034C0340034C0340034C0340034C034EF
:101160000034C0340034C0340034C0340034C034DF
:101170000034C0340034C0340034C03400340F3480
:1011800030341B34C03400340034003400340034B4
:101190000C3400340034003400340034C0340034E3
:1011A000003400340034003403340034003400349C
:1011B00000340034C03400340034003400340034CF
:1011C0000034C0340034003400340034C0340034FF
:1011D000003400340034003400343034003400343F
:1011E00000340034C034003400340034003400349F
:1011F00000340C340034003400340034C034003483
:10120000003400340034003400340334003400343B
:1012100000340034C034003400340034003400346E
:10122000C03400340034003400340034003400345E
:10123000003400340C340034C03400340034003442
:1012400000340034003400340034003403340034FB
:10125000C03400340034003400340034003400342E
:10126000003400340034C034C0340034003400345E
:10127000003400340034003400340034003430349E
:10128000C0340034003400340034003400340034FE
:101290000034003400340C34C034003400340034E2
:1012A00000340034C03400340034003400340334DB
:1012B000C03400340034003400340034C03400340E
:1012C0000034003400340034123404340C34FF345D
:1012D000FF34C0340034C0340034FF34FF34C03431
:1012E0000034C0340034FF34FF34C0340034C03420
:1012F0000034FF34FF34C0340034C0340034C03410
:101300000034FF34FF34C0340034C0340034FF34C0
:10131000FF34C0340034C0340034FF34FF34C034F0
:101320000034C0340034FF34FF34C0340034C034DF
:101330000034C0340034FF34FF34C0340034C034CF
:101340000034FF34FF34C0340034C0340034FF3480
:10135000FF34C0340034C0340034FF34FF3412345E
:1013600004341834FC340034FF34FC34C0347F348B
:10137000F8340034FF34F834C034FF34F03401342E
:10138000FF34F034C134FF34E0340334FF34E0344C
:10139000C334FF34C0340734FF34C034C734FF349F
:1013A000C0340F34FF348034CF34FF34C0341F34A2
:1013B000FF340034DF34FF34C0343F34FE340034B3
:1013C000FF34FE34C0347F34FC340034FF34FC344A
:1013D000C034FF34F8340034FF34F834C134FF34FF
:1013E000F0340134FF34F034C334FF34E0340334D8
:1013F000FF34E034C734FF34C0340734FF34C03422
:10140000CF34FF34C0340F34FF348034DF34FF3442
:10141000C0341F34FF340034FF34FE34C0343F3452
:10142000FE340034FF34FC34C0347F34FC340034E8
:10143000FF34F834C034FF34F8340034FF34F0346F
:10144000C134FF34F0340134FF34E034C334FF34AA
:10145000E0340334FF34C034C734FF34C0340734BD
:10146000FF348034CF34FF34C0340F34FF340034C1
:10147000DF34FF34C0341F34FE340034FF34FE3414
:10148000C0343F34123404341934C0340034FF34CF
:10149000FC34C0347F34C0340034FF34FC34C034F6
:1014A0007F34C0340034FF34F834C034FF34C034E7
:1014B0000034FF34F034C134FF34C0340034FF341E
:1014C000E034C334FF34C0340034FF34C034C73494
:1014D000FF34C0340034FF348034CF34FF34C034A0
:1014E0000034FF340034DF34FF34C0340034FE34C1
:1014F0000034FF34FE34C0340034FC340034FF3494
:10150000FC34C0340034F8340034FF34F834C034D0
:101510000034F0340134FF34F034C0340034E034AB
:101520000334FF34E034C0340034C0340734FF34B3
:10153000C034C0340034C0340F34FF348034C0347D
:101540000034C0341F34FF340034C0340034C0349D
:101550003F34FE340034C0340034C0347F34FC34B3
:101560000034C0340034C034FF34F8340034C034A4
:101570000034C134FF34F0340134C0340034C33497
:10158000FF34E0340334C0340034C734FF34C03493
:101590000734C0340034CF34FF34C0340F34C03487
:1015A0000034DF34FF34C0341F34C0340034FF341F
:1015B000FE34C0343F34123411344934C834073453
:1015C000C0340034C0340734CC340334C034003465
:1015D000C0340334CE340134C0340034C034013458
:1015E000CF340034C0340034C0340034C7348034C5
:1015F000C0340034C0340034C334C034C034003488
:10160000C0340034C134E034C0340034C034003459
:10161000C034F034C0340034C0340034C0347834C2
:10162000C0340034C0340034C0343C34C0340034DE
:10163000C0340034C0341E34C0340034C0340034EC
:10164000C0340F34C0340034C0340034C8340734DC
:10165000C8340034C0340034CC340334CC340034C7
:10166000C0340034CE340134CE340034C0340034BD
:10167000CF340034CF340034C0340034C734803425
:10168000C7348034C0340034C334C034C334C034AD
:10169000C0340034C134E034C134E034C0340034E8
:1016A000C034F034C034F034C0340034C034783442
:1016B000C0347834C0340034C0343C34C0343C349A
:1016C000C0340034C0341E34C0341E34C03400343E
:1016D000C0340F34C0340F34C0340034C034073445
:1016E000C8340734C0340034C0340334CC34033439
:1016F000C0340034C0340134CE340134C03400343A
:10170000C0340034CF340034C0340034C03400342A
:10171000CF340034C0340034C0340034C734803493
:10172000C0340034C0340034C334C034C034003456
:10173000C0340034C134E034C0340034C034003428
:10174000C034F034C0340034C0340034C034783491
:10175000C0340034C0340034C0343C34C0340034AD
:10176000C0340034C0341E34C0340034C0340034BB
:10177000C0340F34C0340034C0340034C8340734AB
:10178000C8340034C0340034CC340334CC34003496
:10179000C0340034CE340134CE340034C03400348C
:1017A000CF340034CF340034C0340034C7348034F4
:1017B000C7348034C0340034C334C034C334C0347C
:1017C000C0340034C134E034C134E034C0340034B7
:1017D000C034F034C034F034C0340034C034783411
:1017E000C0347834C0340034C0343C34C0343C3469
:1017F000C0340034C0341E34C0341E34C03400340D
:10180000C0340F34C0340F34C0340034C034073413
:10181000C8340734C0340034C0340334CC34033407
:10182000C0340034C0340134CE340134C034003408
:10183000C0340034CF340034C0340034C0340034F9
:10184000C7348034C0340034C0340034C334C034AE
:10185000C0340034C0340034C134E034C034003407
:10186000C0340034C034F034C0340034C0340034E8
:10187000C0347834C0340034C0340034C0343C3414
:10188000C0340034C0340034C0341E34C03400349A
:10189000C0340034C0340F34C8340034C03407348A
:1018A000C8340734CC340034C0340334CC3403346B
:1018B000CE340034C0340134CE340134CF3400345B
:1018C000C0340034CF340034C7348034C0340034E2
:1018D000C7348034C334C034C0340034C334C0345B
:1018E000C134E034C0340034C134E034C034F034A6
:1018F000C0340034C034F034C0347834C0340034E0
:10190000C0347834C0343C34C0340034C0343C3447
:10191000C0341E34C0340034C0341E34C0340F34DC
:10192000C0340034C0340F341034FF3403341F3457
:1019300000340134FC340B34003410345034063499
:101940000134C03401340034013430340134003403
:1019500001340C34083400341034503412348E34D2
:1019600040340E3480348E34C0340E3480348E349F
:1019700040340E3400342E3404340E3408342E3403
:101980000C340E3408342E3404340E3400344E3407
:1019900010340E3420344E3430340E3420344E346F
:1019A00010340E3400341034503412344C3450346B
:1019B0008C34A0344C34F0348C34A0344C34503457
:1019C0008C3400342C3444348C3488342C34CC346F
:1019D0008C3488342C3444348C3400344C341434F7
:1019E0002C3428344C343C342C3428344C341434C7
:1019F0002C3400340F34303403340F34FF340034CB
:101A0000003400340034003400340F34FF34003428
:101A1000003400340034003400340F34FF340F3409
:101A2000FF340434CF34FF34003400340034003445
:101A3000C03400340F34FF3400340034C034003478
:101A4000003400340F34FF34C03400340034003428
:101A5000003400341034803406348134C0348B3484
:101A60000034413430344B34003421340C342B34C2
:101A700000341034103406348234C0348C340034D2
:101A8000423430344C34003422340C342C3400349E
:101A90001034603406348134C0348C340034413422
:0E1AA00030344C34003421340C342C340034F7
:020000040001F9
:02000E008C3F25
:02001000323F7D
:02001200FF1FCE
:02E000000034EA
:00000001FF
